:0E00000027C0FECFFDCFFCCFFBCFFACFF9CF4C
:10000E00F8CFD4C2F6CFF5CFF4CFF3CFF2CFF1CFF6
:10001E00F0CFEFCFEECFEDCF1027E80364000A004C
:10002E00010000100001100001000000000000009F
:10003E0000000000010002003800080004003A0031
:10004E000000F894EE27ECBBF1E0FBBFEBBFE5BF81
:10005E00F8E1F1BDE1BD8DE0A2E0BB27ED938A95FD
:10006E00E9F780E094E0A0E6ED930197E9F7E2E48A
:10007E00F0E085919591009761F0A591B59105906D
:10008E001590BF01F00105900D920197E1F7FB016C
:10009E00F0CFEFE5EDBFE4E0EEBFC8E2D1E0C4C3C0
:1000AE00E881EFB9779BFECFEFB1219608952297A5
:1000BE00C298EFEFEA93F4DFEE81E064EA93F0DFAB
:1000CE00EC81FD81E883F983E981EA93E9DFE88138
:1000DE00EA93E6DFEA81FB81E883F983E981EA931B
:1000EE00DFDFE881EA93DCDFE5E9EA93D9DFEFEFC2
:1000FE00EA93D6DF2796089596D40FEF1FEF3FEFC2
:10010E003F3F19F40150104009F405C0EFEFEA9398
:10011E00C7DF3E2FF5CFE32F8BD46FC084D40FEF04
:10012E001FEF3FEF3E3F19F00150104009F405C09C
:10013E00EFEFEA93B5DF3E2FF5CFE32F79D45DC015
:10014E001A9310E01A3028F4EFEFEA93A9DF1F5F3D
:10015E00F9CFC29A18C169D4E1E1EA93AD81BE81AB
:10016E008F819885E7E03AD4FA93EA93AF81B88508
:10017E00E9E02BD4FA93EA939ADFD0DFEE3F21F039
:10018E00DFDFEFEFFFEF9FC000E010E00030E1E0B7
:10019E001E0788F4EA81FB813196EA83FB8331974F
:1001AE00FF93EF93EFEFEA937BDFAF91BF91EC9369
:1001BE000F5F1F4FEBCF85C038D400E010E000304A
:1001CE00E1E01E0788F4EA81FB813196EA83FB8326
:1001DE003197FF93EF93EFEFEA9362DFAF91BF9109
:1001EE00EC930F5F1F4FEBCFEFEFEA9359DFEFEF7B
:1001FE00EA9356DFE0E0F0E01DD4249608952497AC
:10020E00EFEFE883E983E0E0EA83EB83EFEFEA9335
:10021E0047DFAE2FEC81EA1749F0ECD331976040FF
:10022E007040EDD3DF01CB01F8D308F001C0EECF63
:10023E00E1D3EFD319F4E1E0F0E002C0E0E0F0E04A
:10024E0025960895F2D3E8E1EA93AD81BE818F81C0
:10025E009885E7E0C3D3FA93EA93AF81B885E9E0D6
:10026E00B4D3FA93EA9323DFE0E0EA93C8DFE130F8
:10027E00A0E0FA0721F464DFEFEFFFEF24C0EEEF0A
:10028E00EA930EDF00E010E00030E2E01E0750F4CB
:10029E00AA81BB81ED91AA83BB83EA9301DF0F5F35
:1002AE001F4FF2CFEFEFEA93FBDEEFEFEA93F8DEAC
:1002BE00EFEFEA93F5DEEF70E53019F0EFEFFFEFB9
:1002CE0002C0E0E0F0E0B6D328960895AED3E8B3CE
:1002DE00E77DE8BBC49AE7B3E862E7BBC29ABA9A75
:1002EE00B89AE0E5EDB9E1E0EEB900E010E00A30D1
:1002FE00E0E01E0734F4EFEFEA93D2DE0F5F1F4FFC
:10030E00F6CFE0E0EA93E0E0F0E0FA93EA93FA93B6
:10031E00EA93CDDEF1DEE13019F012DFE1E044C107
:10032E000FEF1FEFEFEFEA93BBDEE03019F0015055
:10033E00104009F40AC0E1E0EA93E0E0F0E0FA933D
:10034E00EA93FA93EA93B3DEEDCFFADE002E012A9A
:10035E0011F4E2E029C1E0E027C11A93E4E6F2E0ED
:10036E008E169F0680F414B115B1F401E85DFE4FB0
:10037E001083F40131964F01E0E0F2E0E815F90543
:10038E0011F4689420F8199108954FD3E89420F849
:10039E00A0918C03B0918D0380918E0390918F0369
:1003AE00AB32EFEDBE07EDE28E07E0E09E0748F0C0
:1003BE00E0E0E0938C03E0938D03E0938E03E093F3
:1003CE008F03E0918C03F0918D0360918E037091F9
:1003DE008F031AD3E8E2F1E0FA93EA9333DF309712
:1003EE0039F092989398EFEF6E1608F46394DCC090
:1003FE00F894E0E0F2E0E815F905D0F400E012E040
:10040E000815190580F4F801E050F240E85DFE4F42
:10041E000F01A8E2B1E0A00FB11FEC91D001EC9357
:10042E000F5F1F4FEDCFF801EF5FF1404F0102C09C
:10043E008824992478946624F50131965F01E09121
:10044E008C03F0918D0360918E0370918F03EF5F9B
:10045E00FF4F6F4F7F4FE0938C03F0938D036093AC
:10046E008E0370938F03689421F89EC023FC06C000
:10047E00A8E2B1E0A80DB91DEC9104C0F401E85D4D
:10048E00FD4FE081EABD26FE05C0A0E024FCA1E000
:10049E00A03009F011C0E89426F823FC03C068943C
:1004AE0022F806C0E89422F800240A140B0420F463
:1004BE00689424F8E89425F8EFEFF0E0E815F905D4
:1004CE0089F4689426F88824992423FC01C001C07D
:1004DE00E89423F8E1E0F0E0AE16BF0610F4E7E092
:1004EE007E2E03C0F40131964F0108959ED2A09145
:1004FE009003B09191038091920390919303AB324C
:10050E00EFEDBE07EDE28E07E0E09E0748F0E0E07B
:10051E00E0939003E0939103E0939203E0939303AF
:10052E0022FC11C0929AE0919003F0919103609198
:10053E0092037091930368D2E8E2F1E0FA93EA93A2
:10054E000ADE8F0122C09298E8E2F2E0FA93EA9373
:10055E0033DE8F01E0919003F0919103609192034D
:10056E0070919303EF5FFF4F6F4F7F4FE0939003B8
:10057E00F0939103609392037093930300240A14F3
:10058E000B0418F4F50131975F01002E012A21F4B6
:10059E00689425F8662406C092989398EFEF6E162D
:1005AE0008F46394E89424F848D208950A921A92B3
:1005BE00FA926A937A938A939A93AA93BA93EA9346
:1005CE00FA93EFB7EA93FF245394E4E0E51561F450
:1005DE005524E1E0E71519F0E3E0E71509F4BDDE77
:1005EE00E6E0E71509F442DFE1E0E51509F00EC19A
:1005FE004394EAE2E41541F54424B7990DC0E0E0D6
:10060E00E0939603A0919703AF3F28F4E0919703F0
:10061E00EF5FE09397030CC0E0E0E0939703A091A7
:10062E009603AF3F28F4E0919603EF5FE0939603B5
:10063E00A0919603AB3010F0689427F8A091970321
:10064E00A63010F0E89427F8EEE1E41509F07BC02F
:10065E0027FE3CC0E0E0E71531F4E61521F420FC5E
:10066E0002C021FE01C017C09598E1E07E2E8824BD
:10067E009924AA24BB24E0918C03F0918D03609100
:10068E008E0370918F03E0939003F0939103609328
:10069E00920370939303E3E0E71511F4E1E07E2EED
:1006AE00E1E0E71549F4EEE6F3E0EA15FB0520F488
:1006BE0020FC02C021FE01C008C0E4E07E2EE894BA
:1006CE0022F8689424F8E89425F83DC0E1E0E71597
:1006DE0041F46501E0E0E0939403E0939503E3E0D9
:1006EE007E2EE2E0E71511F46894F0F8E3E0E715EA
:1006FE00B1F4E0919403F09195033196E093940355
:10070E00F0939503A0919403B0919503A035E1E089
:10071E00BE0728F0F60132965F016894F0F8F0FEFD
:10072E0012C0E0E1F0E0EA15FB0518F4E0E0E61592
:10073E0009F008C0E4E07E2E689424F8E89422F8CC
:10074E0025F801C07724E3E2E41509F051C0E4E096
:10075E00E71511F425FC01C00EC088249924689475
:10076E0026F8E89423F8E5E07E2EE0E0E093980387
:10077E00E0939903959AE5E0E71599F4E0919803D3
:10078E00F09199033196E0939803F0939903A09119
:10079E009803B0919903A838E0E0BE0710F0E6E0A8
:1007AE007E2EE7E0E71571F4EFE7EABDE0E0E093B7
:1007BE009603E0939703E8E07E2EE0E0E093940347
:1007CE00E0939503E8E0E71599F4E0919403F09136
:1007DE0095033196E0939403F0939503A0919403BF
:1007EE00B0919503A536E0E0BE0710F095987724FA
:1007FE00772061F4F50131965F01E4ECF9E0EA153A
:10080E00FB0521F4AA24BB24E9E07E2EE991EFBF7B
:10081E00F991E991B991A9919991899179916991FA
:10082E00F990199009901895FF2410E0EFEFE1BFB1
:10083E00E0E0E8BBE2E0E7BBE0E0E5BBE4BBE2BB47
:10084E00ECE2E1BBE0E0E3BFE2BFE1E8EFBDE9E0EF
:10085E00EEBDE0E0EDBDECBDE7BDE6BDEBBDEABD36
:10086E00E9BDE8BDE2BDE5BDE4BDE3BDE5BFE4E045
:10087E00E9BFE0E8E8B9E0E0E0BFE0E6E7B9E5EEC1
:10088E00E6B9E0E6E7B9369AE9E07E2E7894929AD8
:10089E00939AEFE7EABDE0EDF7E0FA93EA9389D099
:1008AE009398959AE0EDF7E0FA93EA9382D09298B6
:1008BE0093989598E4EFF1E0FA93EA937AD006DDF7
:1008CE00E03031F0E4E6F0E0FA93EA9372D0F7CF3D
:1008DE00EAE2FFED6DE270E097D0E8E2F1E0FA9324
:1008EE00EA9339DC309749F4E8E2F1E0FA93EA93BF
:1008FE0063DC939A929A6624772421FE09C0EFEF67
:10090E00EA93CEDBE03019F0E89421F8929807C014
:10091E0020FE03C03ADD929A02C024FCE7DD772068
:10092E00A1F4E0E0E41511F4F0FC01C009C0E89474
:10093E00F0F81F5F1F3709F4929A1F3F09F492983F
:10094E00E1E0E41511F46894F0F8E9E0E715C9F474
:10095E00EAE2FFED6DE270E057D0E8E2F1E0FA93E3
:10096E00EA93F9DB309719F0EFEF6E2E0AC0E8E24A
:10097E00F1E0FA93EA9320DC77246624E89421F8D8
:10098E0020F8E4E1E61598F4E9E07E2E929893982B
:10099E0095989CDCE03031F0E8ECF0E0FA93EA93C5
:1009AE0008D0F7CF929AE89421F820F824F8A5CF32
:1009BE00FFCFE991F991309639F080ED97E00197EC
:1009CE00F1F7A8953197C9F70895EE230E2EFD0184
:1009DE0021F0EE0FFF1F0A94E1F70895EE230E2E7D
:1009EE00FD01BC0131F076956795F795E7950A9470
:1009FE00D1F70895E881F9816A817B810895E883B2
:100A0E00F9836A837B8308957A936A93FA93EA93C0
:100A1E000895309760407040089500240A160B0622
:100A2E000806090608953A932A931A930A9308958D
:100A3E003B812A81198108810895099119910895A0
:00000001FF
